:020000040800F2
:100000006009002045010008B9100008211000080F
:10001000B5100008B10100085F2C000800000000C6
:100020000000000000000000000000002523000880
:10003000B10D000800000000251D00087125000812
:100040005F0100085F0100085F0100085F01000810
:100050005F0100085F0100085F0100085F01000800
:100060005F0100085F0100085F0100085F010008F0
:100070005F0100085F0100085F0100085F010008E0
:100080005F0100085F0100085F0100085F010008D0
:100090005F0100085F0100085F0100085F010008C0
:1000A0005F0100085F0100085F0100085F010008B0
:1000B0005F010008D52500085F0100085F01000806
:1000C0005F0100085F0100085F0100085F01000890
:1000D0005F010008B527000811280008F52800086E
:1000E0005F0100085F0100085F0100085F01000870
:1000F0005F0100085F0100085F0100085F01000860
:100100005F0100085F0100085F0100085F0100084F
:100110005F0100085F0100085F0100085F0100083F
:100120005F0100085F0100085F0100085F0100082F
:10013000DFF80CD000F02AF800480047392F0008FB
:10014000600900200648804706480047FEE7FEE7B2
:10015000FEE7FEE7FEE7FEE7FEE7FEE7FEE7FEE777
:100160007525000831010008D2B201E000F8012B2A
:10017000491EFBD270470022F6E710B513460A4627
:1001800004461946FFF7F0FF204610BD064C074D08
:1001900006E0E06840F0010394E807009847103457
:1001A000AC42F6D3FFF7C8FFE03200080033000886
:1001B00000BFFEE710B502460B460020002104E018
:1001C000545C0444E0B24C1CE1B29942F8DBC443F5
:1001D000E0B2441CE0B210BDFEB5002000900190DA
:1001E000029000F037FF414800780A281DD14048AE
:1001F000007840490978884217D13D4840783D4908
:100200004978884211D13A48007A3A49097A8842B5
:100210000BD13748407A3749497A884205D1364868
:10022000008840F40040344908803348008800F4D6
:100230000040002858D0012002F0E8FD00202F499E
:10024000087048708870C87008712D49087048702F
:100250008870C87008712B49087048708870C87021
:1002600008712949087048708870C870087100F0DA
:10027000F1FE0020224908701D48007948701C4892
:10028000407988701A488079C8701948C079087117
:1002900000201E4908701A48407848701848807835
:1002A00088701748C078C870154800790871012017
:1002B00001F0CAF812484078040611488078050415
:1002C0000F48C0780602601930440D490979471873
:1002D00001200F49087000F0BDFE00F0BBFE0020B9
:1002E0000249087004490880FEBD00000900002092
:1002F000D80100200C0000200A0000202C00002063
:100300001600002034000020390000201B000020CF
:100310004100002010B588B07F480078012838D10E
:1003200000207D490870FC207C490870112048702D
:100330007B48007888707A484078C8707848807820
:1003400008717748C078487175480079887107212D
:100350007248FFF72FFF7149C8710020714908608A
:10036000FF22E121012001F02BFC08236B4AA82188
:10037000012001F0E7FB012001F066F801206A4945
:10038000C1F8A4016949087000206949088000F09B
:1003900061FE6748008840F6B83188427BDC00F097
:1003A00059FE604884380068002857D100F052FE9A
:1003B0006946012001F0A4FB0446204602F000F843
:1003C0005CA002F007F804F040004028EDD10020C6
:1003D0008DF80A000721684600F0EBFC55A001F0FB
:1003E000F9FF9DF801004E490978884254D19DF8E3
:1003F00002004B49497888424ED19DF80300484994
:100400008978884248D19DF804004549C9788842D6
:1004100042D19DF805004249097988423CD14348C0
:10042000007801281BD141480078401C3F490870E2
:1004300012203A49487007213848FFF7BBFE374978
:10044000C8710020374908600823344AA8210120D8
:1004500001F078FB01203449C1F8A40158E00020E4
:10046000324908700E21344800F0A3FC31A001F09D
:10047000B1FF32480178012001F040F810202E49E8
:1004800048700E212C4801F08FFF2DA001F0A2FF33
:10049000012008B010BD16E000202249086011209C
:1004A0001E49487007211D48FFF784FE1B49C8718B
:1004B00008230A46A821012001F044FB01201A4923
:1004C000C1F8A40124E00020154908704870887024
:1004D000C87008711B49087048708870C87008712E
:1004E0001949087048708870C870087117490870F9
:1004F00048708870C870087130200F4948700E210C
:100500000D4801F051FF12A001F064FF0120C0E787
:1005100000F0A0FD0020BCE73E00002042000020CB
:100520002C000020A4812142008021428200002072
:10053000200000200A000000CC0300202A00002038
:100540004F4B0A00390000201B000020160000203D
:10055000333030300A00000010B588B03C480088C5
:1005600040F2DC51884268DA3A480068002861D1DC
:1005700000F070FD6946012001F0C2FA044604F063
:100580004000402856D100208DF80A000721684617
:1005900000F00FFC30A001F01DFF9DF8010078B9BC
:1005A0009DF8020060B99DF8030048B900202B496E
:1005B000087048708870C8700871012008B010BDBC
:1005C0002748007807280FD10020244908709DF89B
:1005D000000048709DF8010088709DF80200C87006
:1005E0009DF80300087123E01D480078082810D109
:1005F0009DF80100194908709DF8020048709DF8A7
:10060000030088709DF80400C8709DF8050008710B
:100610000EE00020114908709DF8010048709DF817
:10062000020088709DF80300C8709DF804000871EE
:100630000120C3E700F00EFD08E000200749087024
:1006400048708870C87008710120B7E70020B5E7CE
:1006500032000020208121420A00000039000020E1
:100660002A0000203EB5002000900190029000F08A
:10067000F1FCFE480078082829D1FD48007875284B
:1006800025D1FB484078702821D1F948807864282A
:100690001DD1F748C078612819D1F5480079742830
:1006A00015D1F3484079652811D10020EF49087031
:1006B00000BFF048006800F4E060EF490843001D07
:1006C000EC490860BFF3408F00BF00BFFEE7E84879
:1006D0000078752807D0E6480078FA2803D0002073
:1006E000E24908703EBDE14800780E2800DAF9E7DB
:1006F000DE480078401EDE49085CFB2800D0F1E7A8
:10070000DB48807AA02804D1D8480078152800D08A
:10071000E8E7D64800780E281ED1D5480078FA2898
:1007200014D1D348407BFB2810D1D448008840F432
:100730000040D24908800020CC4908700E21CC48E6
:1007400000F037FBCEA001F045FE4AE00020C7498B
:100750000870CA49088044E0C448007815281ED1B2
:10076000C3480078FA2814D1C148007DFB2810D175
:10077000C248008840F40040C04908800020BB49BE
:1007800008701521BA4800F014FBBDA001F022FE4C
:1007900027E00020B5490870B849088021E0B34837
:1007A000007811281DD1B2480078FA2814D1B04839
:1007B000007CFB2810D1B148008840F40040AF49CC
:1007C00008800020A94908701121A94800F0F1FA19
:1007D000ABA001F0FFFD04E00020A4490870A74988
:1007E0000880A648008800F40040002871D000F07E
:1007F00031FC9F488079A34988719D48C179A148FF
:10080000C1719B48017A9F4801729948417A9D487D
:1008100041729748807A9B498872084680799A4944
:1008200088719848C1799848C1719648017A96486C
:1008300001729448417A944841729248807A94288F
:100840004CD018DC732834D00CDC252825D004DCEF
:1008500021281AD022287DD11BE0262821D07128FA
:10086000F9D122E0742828D075282AD078282CD0F5
:100870008228F0D12EE0A03809286BD2DFE800F002
:10088000329CA0F5F4F3F2F1F00000207D4988726B
:10089000CBE100207B498872C7E10020794988724A
:1008A000C3E1002077498872BFE100207549887252
:1008B000BBE1002073498872B7E10020714988725A
:1008C000B3E100206F498872AFE100206D49887262
:1008D000ABE1AEE100206B498872A6E100206949D6
:1008E0008872A2E1002061490870664880796749F2
:1008F00088716448C1796548C1716248017A63486A
:1009000001726048417A614841725E48807A5F496D
:1009100088725748407B5B4948735548817B5948EA
:1009200081735348C17B5748C1735148017C554876
:1009300001744F48417C534841744D48407B5449B1
:1009400008704B48807B48704948C07B8870484895
:10095000007C00E068E1C8704548407C08710120D7
:100960004C49087000204C490880012000F06CFDC3
:100970004AA001F02FFD04E0FFF7CCFC044604B1CF
:1009800000E0F9E700BF45A001F024FD0020454943
:10099000087048708870C8700871434908704870C2
:1009A0008870C87008714149087048708870C870B4
:1009B00008713449887238E100203249887234E184
:1009C0003948407848B93848807830B93648C078D6
:1009D00018B93548007900B927E10020234908708B
:1009E00028488079324988712648C1793048C171D8
:1009F0002448017A2E4801722248417A2C484172DB
:100A00002048807A2A4988720120C872062008731B
:100A10000020487324480178254881732248417892
:100A20002348C17320488178214801741E48C17849
:100A30001F4841741C4801791D488174162101F03A
:100A4000B3FC322002F0E2F91621194800F0B1F9A6
:100A50000BA001F0BFFC002013490870487029E08A
:100A600099E0DDE0D8E0D3E02BE029E003000020AE
:100A7000100100200CED00E00000FA050400002049
:100A80000A00000004030020A0020020CC03002084
:100A90002C0000203E0000202000002030303030AC
:100AA0000A000000390000201B0000201600002072
:100AB000680300208870C87008715F498872B4E0CC
:100AC000B3E000205D4908705D480178012000F026
:100AD00015FD00205B4908805BA001F07BFC04E071
:100AE000FFF73AFD044604B100E0F9E700BF56A065
:100AF00001F070FC50488079554988714E48C179A1
:100B00005348C1714C48017A514801724A48417AB0
:100B10004F4841724848807A4D4988720120C87216
:100B200006200873002048734A48017848488173BA
:100B3000484841784648C173464881784448017422
:100B40004448C17842484174424801794048817420
:100B5000162101F029FC322002F058F916213C48F8
:100B600000F027F939A001F035FC00203949087060
:100B700048708870C870087137490870487088706C
:100B8000C87008713549087048708870C87008715D
:100B90002949887249E03248407B29490870264833
:100BA0008079304988712448C1792E48C171224822
:100BB000017A2C4801722048417A2A4841721E4825
:100BC000807A28498872012048700E21254801F05A
:100BD000EBFB322002F01AF919480078224908800C
:100BE00001F0AAFB00201B49087048708870C8708B
:100BF00008711949087048708870C87008711749E1
:100C0000087048708870C87008710B4988720CE0D1
:100C100000200949887208E000200749887204E032
:100C200000200549887200E000BF00BF00200F4986
:100C3000088000BF56E500000403002003000020E8
:100C40002A00002032000020343434340A0000002E
:100C500068030020390000201B000020160000203F
:100C6000100100203004002038050020040000207E
:100C7000FA204A490870102048700020887000212E
:100C80004648C170017141710020444988710021BA
:100C90004248C1710172417200204049C87400216C
:100CA0003E480175FB203D494875FA203C490870D3
:100CB000102048700020887000213948C1700171EF
:100CC000417100203649887100213548C171017297
:100CD00041720020324981F84B000021304880F8F1
:100CE0004C10FB202E4981F84D00FA202D49087048
:100CF000102048700020887000212A48C1700171BE
:100D0000417100202749887100212648C171017274
:100D1000417200202349C872002122480173FB2040
:100D200020494873FA20204908701020487000209C
:100D3000887000211C48C1700171417100201A495E
:100D4000887100211848C171017241720020164952
:100D5000C874002114480175FB2013494875FA2016
:100D600012490870102048700020887000210F4838
:100D7000C1700171417100200C49887100210B483C
:100D8000C1710172417200200849C87200210748F0
:100D90000173FB200549487370470000A002002042
:100DA000040300203004002068030020CC0300204E
:100DB00070472DE9F04104460E460DE025782811D4
:100DC00000F030F9074601F0FBFA284600F02AF956
:100DD000074601F0F5FA641C3000A6F10101CEB21D
:100DE000ECD1BDE8F081000030B5044604254FF495
:100DF000302000F06FF80546042D17D10C4800692B
:100E000040F002000A49086108464461006940F068
:100E1000400008614FF4302000F05CF805460448BB
:100E2000006941F6FD71084001490861284630BD5E
:100E30000020024004200B49C96801F0010109B1FA
:100E400001200EE00749C96801F0040109B1022040
:100E500007E00449C96801F0100109B1032000E06E
:100E600004207047002002400348006940F08000E1
:100E700001490861704700000020024070B5044637
:100E80000D460426F00200F025F80646042E11D186
:100E90000948006940F00100074908612580F00217
:100EA00000F018F806460448006941F6FE71084053
:100EB00001490861304670BD0020024002480349E4
:100EC000486003484860704723016745002002409E
:100ED000AB89EFCD00B502460423FFF7ABFF034615
:100EE00003E0FFF7A7FF0346521E012B01D1002AA2
:100EF000F7D102B90523184600BD2DE9F04102469D
:100F000000250026002000230024002791F803C0BC
:100F10000CF00F0591F803C00CF0100CBCF1000FA1
:100F200003D091F802C04CEA050591F800C0BCF16D
:100F3000000F31D0146800202BE04FF0010C0CFAA8
:100F400000F3B1F800C00CEA03069E4220D18300F2
:100F50004FF00F0C0CFA03F7BC4305FA03FC4CEA04
:100F6000040491F803C0BCF1280F06D14FF0010C26
:100F70000CFA00FCC2F814C00AE091F803C0BCF1FE
:100F8000480F05D14FF0010C0CFA00FCC2F810C05C
:100F9000401C0828D1D31460B1F800C0BCF1FF0F89
:100FA00034DD546800202EE000F1080C4FF00108F9
:100FB00008FA0CF3B1F800C00CEA03069E4221D1F6
:100FC00083004FF00F0C0CFA03F7BC4305FA03FC47
:100FD0004CEA040491F803C0BCF1280F05D100F1DC
:100FE000080C08FA0CF8C2F8148091F803C0BCF1A0
:100FF000480F07D100F1080C4FF0010808FA0CF86F
:10100000C2F81080401C0828CED35460BDE8F0819F
:10101000416170470161704701460A8890B270478C
:1010200000BFFEE70146002001F00F02092A04DCA0
:1010300001F00F0202F1300003E001F00F0237323D
:10104000D0B270474CF6CC400149086070470000B0
:101050000030004010B500F013F810BD70B5054623
:101060000C4645F2555000F01FF8284600F010F8E5
:10107000204600F013F800F003F8FFF7E3FF70BD1F
:101080004AF6AA200149086070470000003000407D
:101090000149486070470000003000400149886005
:1010A00070470000003000400149086070470000B0
:1010B0000030004000BFFEE7704700007CB50546E9
:1010C00012A103C9CDE900010821284601F002F967
:1010D00005236A463021284600F034FD05236A4680
:1010E0001021284600F09EFC002406E01DF80400B4
:1010F000A52800D003E0601CC4B2052CF6DB00BFBD
:10110000052C01D001207CBD0020FCE7A5A5A5A5EC
:10111000A500000008B501211C2000F015FE4020AC
:10112000ADF8000010208DF8030003208DF80200B8
:1011300069463048FFF7E1FE40212E48FFF76AFF7D
:101140001020ADF8000069462B48FFF7D6FE1021AD
:101150002948FFF75FFF0120ADF8000048208DF817
:10116000030003208DF8020069462348FFF7C5FEFF
:101170004FF40070ADF8000010208DF8030003203C
:101180008DF8020069461B48FFF7B7FE4FF4007167
:101190001848FFF73FFF4FF48050ADF80000694654
:1011A0001448FFF7AAFE4FF480511248FFF732FFB0
:1011B0004FF48070ADF8000048208DF80300032044
:1011C0008DF8020069460B48FFF797FE00F0B0FF6C
:1011D00000F06CFF00200949086001200849C1F8AF
:1011E0009001002005490C31086001200549C1F833
:1011F000B00108BD000C0140000801409881214267
:10120000000021420080214210B504460222232121
:10121000204600F0D5FC05231E4A2A21204600F076
:1012200091FC05231B4A3021204600F08BFC3F2215
:101230002121204600F0C4FC01222221204600F09A
:10124000BFFC1A222521204600F0BAFC24222621C8
:10125000204600F0B5FC0F222021204600F0B0FC13
:101260000A223121204600F0ABFC01223D2120461C
:1012700000F0A6FC00223C21204600F0A1FC7022D8
:101280002721204600F09CFCFF22E221204600F0AE
:1012900097FC10BDC132000810B50446022223217C
:1012A000204600F08DFC05231E4A2A21204600F02E
:1012B00049FC05231B4A3021204600F043FC3F2215
:1012C0002121204600F07CFC01222221204600F052
:1012D00077FC12222521204600F072FC04222621F0
:1012E000204600F06DFC0F222021204600F068FC13
:1012F0000A223121204600F063FC01223D212046D4
:1013000000F05EFC00223C21204600F059FC7022D7
:101310002721204600F054FCFF22E221204600F065
:101320004FFC10BDB232000810B504460222232142
:10133000204600F045FC05231E4A2A21204600F0E5
:1013400001FC05231B4A3021204600F0FBFB302224
:101350002121204600F034FC01222221204600F009
:101360002FFC12222521204600F02AFC21222621D2
:10137000204600F025FC0F222021204600F020FC12
:101380000A223121204600F01BFC00223D2120468C
:1013900000F016FC01223C21204600F011FC7022D6
:1013A0002721204600F00CFCFF22E221204600F01D
:1013B00007FC10BDA332000810B50446012223210A
:1013C000204600F0FDFB05231E4A2A21204600F09E
:1013D000B9FB05231B4A3021204600F0B3FB302225
:1013E0002121204600F0ECFB01222221204600F0C2
:1013F000E7FB19222521204600F0E2FB04222621EA
:10140000204600F0DDFB0F222021204600F0D8FB13
:1014100006223121204600F0D3FB01223D21204647
:1014200000F0CEFB00223C21204600F0C9FB7022D8
:101430002721204600F0C4FBFF22E221204600F0D5
:10144000BFFB10BDD032000810B504461CB9002007
:101450002749086003E0002025490C31086001227B
:101460002321204600F0ACFB0323224A2A212046F8
:1014700000F068FB0323204A3021204600F062FB85
:1014800001222121204600F09BFB0122222120463F
:1014900000F096FB2A222521204600F091FB042231
:1014A0002621204600F08CFB0F222021204600F050
:1014B00087FB06223D21204600F082FB01223C21D1
:1014C000204600F07DFB70222721204600F078FBAB
:1014D000FF22E221204600F073FB1CB901200449E1
:1014E000086003E0012002490C31086010BD0000D3
:1014F00098812142993200089432000870B5044660
:101500000D461CB900202649086003E0002024494C
:101510000C3108600C2D37D2DFE805F0060A0E12F8
:10152000161A1E22262A2E322046FFF7FDFE2BE039
:10153000204600F09FF927E0204600F02BFA23E038
:101540002046FFF7A9FE1FE0204600F003F91BE04C
:10155000204600F06FF817E02046FFF755FE13E035
:10156000204600F0AFF80FE0204600F0CBF90BE08A
:101570002046FFF721FF07E0204600F013F803E0C4
:10158000204600F02FF900BF00BF1CB9012004491C
:10159000086003E0012002490C31086070BD0000C2
:1015A0009881214210B5044602222321204600F0F2
:1015B00007FB04231E4A2A21204600F0C3FA042315
:1015C0001B4A3021204600F0BDFA3022212120465E
:1015D00000F0F6FA01222221204600F0F1FA202242
:1015E0002521204600F0ECFA24222621204600F096
:1015F000E7FA0F222021204600F0E2FA08223121EA
:10160000204600F0DDFA01223D21204600F0D8FA04
:1016100000223C21204600F0D3FA702227212046E8
:1016200000F0CEFAFF22E221204600F0C9FA10BDF8
:10163000D532000810B5044602222321204600F0CE
:10164000BFFA05231E4A2A21204600F07BFA052313
:101650001B4A3021204600F075FA30222121204615
:1016600000F0AEFA01222221204600F0A9FA12224F
:101670002521204600F0A4FA24222621204600F04D
:101680009FFA0F222021204600F09AFA0A223121E7
:10169000204600F095FA01223D21204600F090FA04
:1016A00000223C21204600F08BFA702227212046A0
:1016B00000F086FAFF22E221204600F081FA10BDF8
:1016C000BC32000810B5044601222321204600F058
:1016D00077FA05231E4A2A21204600F033FA052313
:1016E0001B4A3021204600F02DFA302221212046CD
:1016F00000F066FA01222221204600F061FA102251
:101700002521204600F05CFA04222621204600F024
:1017100057FA0F222021204600F052FA06223121EA
:10172000204600F04DFA01223D21204600F048FA03
:1017300000223C21204600F043FA70222721204657
:1017400000F03EFAFF22E221204600F039FA10BDF7
:10175000C632000810B5044602222321204600F0BC
:101760002FFA05231E4A2A21204600F0EBF9052313
:101770001B4A3021204600F0E5F930222121204685
:1017800000F01EFA01222221204600F019FA12224E
:101790002521204600F014FA24222621204600F0BC
:1017A0000FFA0F222021204600F00AFA08223121E8
:1017B000204600F005FA01223D21204600F000FA03
:1017C00000223C21204600F0FBF970222721204610
:1017D00000F0F6F9FF22E221204600F0F1F910BDF9
:1017E000B732000810B5044602222321204600F03B
:1017F000E7F904231E4A2A21204600F0A3F9042316
:101800001B4A3021204600F09DF93022212120463C
:1018100000F0D6F901222221204600F0D1F91C2245
:101820002521204600F0CCF924222621204600F074
:10183000C7F90F222021204600F0C2F908223121E9
:10184000204600F0BDF901223D21204600F0B8F904
:1018500000223C21204600F0B3F9702227212046C7
:1018600000F0AEF9FF22E221204600F0A9F910BDF8
:10187000DA32000810B5044603222321204600F086
:101880009FF905231E4A2A21204600F05BF9052313
:101890001B4A3021204600F055F93F2221212046E5
:1018A00000F08EF93F222221204600F089F92822FB
:1018B0002521204600F084F904222621204600F04C
:1018C0007FF90B222021204600F07AF90A223121EB
:1018D000204600F075F901223D21204600F070F904
:1018E00000223C21204600F06BF97022272120467F
:1018F00000F066F9FF22E221204600F061F910BDF8
:10190000A832000810B5044601222321204600F029
:1019100057F903231E4A2A21204600F013F9032316
:101920001B4A3021204600F00DF9302221212046AB
:1019300000F046F901222221204600F041F92A2236
:101940002521204600F03CF904222621204600F003
:1019500037F90F222021204600F032F907223121E9
:10196000204600F02DF900223D21204600F028F904
:1019700001223C21204600F023F970222721204635
:1019800000F01EF9FF22E221204600F019F910BDF7
:10199000CB32000810B5044603222321204600F074
:1019A0000FF905231E4A2A21204600F0CBF8052313
:1019B0001B4A3021204600F0C5F830222121204664
:1019C00000F0FEF801222221204600F0F9F8102252
:1019D0002521204600F0F4F804222621204600F0BC
:1019E000EFF80F222021204600F0EAF80A223121E8
:1019F000204600F0E5F801223D21204600F0E0F805
:101A000000223C21204600F0DBF8702227212046EE
:101A100000F0D6F8FF22E221204600F0D1F810BDF8
:101A2000AD3200082DE9F0478046894615461E462E
:101A3000B8F1000F16D1002017490860494640460A
:101A400000F0F4FB0746002406E0FF21404600F0CA
:101A5000EDFB2855601CC4B2B442F6DB01200E49F0
:101A6000086015E000200D4908604946404600F036
:101A7000DDFB0746002406E0FF21404600F0D6FBD0
:101A80002855601CC4B2B442F6DB0120034908604B
:101A90003846BDE8F087000090012142B081214224
:101AA00070B505460E4685B90020114908603146DB
:101AB000284600F0BBFBFF21284600F0B7FB044698
:101AC00001200C49C1F890010FE000200A4908608C
:101AD0003146284600F0AAFBFF21284600F0A6FB6D
:101AE000044601200549C1F8B001204670BD000040
:101AF0009001214200002142B08121420080214218
:101B000070B506460D461021304600F0E3FB072174
:101B10003046FFF7C5FF044622462721304600F035
:101B20004FF804F0400050B10A232A4661213046A4
:101B3000FFF778FFFF22E221304600F041F820460F
:101B400070BD00002DE9F0478046894615461E46C7
:101B5000B8F1000F16D100201749086049464046E9
:101B600000F064FB0746002406E015F8011B404620
:101B700000F05CFB601CC4B2B442F6DB01200E49ED
:101B8000086015E000200D4908604946404600F015
:101B90004DFB0746002406E015F8011B404600F007
:101BA00045FB601CC4B2B442F6DB01200349086067
:101BB0003846BDE8F087000090012142B081214203
:101BC0002DE9F04104460E46154684B9002011491E
:101BD00008603146204600F029FB0746294620468A
:101BE00000F024FB01200C49C1F890010FE0002017
:101BF0000A4908603146204600F018FB074629468E
:101C0000204600F013FB01200549C1F8B001384619
:101C1000BDE8F0819001214200002142B0812142C3
:101C20000080214208B54FF4C06000F071F8262012
:101C30008DF8000001208DF8010002208DF80200CF
:101C400001208DF80300684600F02AF827208DF85F
:101C5000000001208DF801008DF802008DF80300CE
:101C6000684600F01DF825208DF8000000208DF852
:101C7000010001208DF802008DF80300684600F095
:101C80000FF81D208DF8000000208DF801008DF860
:101C9000020001208DF80300684600F001F808BD3D
:101CA00070B5002100230F22C47804B3154C2468BA
:101CB00004F4E064C4F5E064210AC1F10403CA40FD
:101CC000447804FA03F184781440214309010E4C4E
:101CD0000678A155047804F01F050124AC4005786E
:101CE0006D11AD0005F1E025C5F8004109E004786B
:101CF00004F01F050124AC40044D0678761145F828
:101D0000264070BD0CED00E000E400E080E100E062
:101D100002490143024A1160704700000000FA05C1
:101D20000CED00E07047000029B1064AD269024379
:101D3000044BDA6104E0034AD2698243014BDA6161
:101D4000704700000010024029B1064A9269024320
:101D5000044B9A6104E0034A92698243014B9A6101
:101D6000704700000010024010B500F033F84FF447
:101D7000803000F0F1F800F04DF90446012C1ED13E
:101D8000002000F0DDF8002000F018F9A00200F0BB
:101D900009F94FF4E011200400F022F9012000F0CD
:101DA00019F900BF392000F0A5F80028FAD0022068
:101DB00000F024F900BF00F0BBF80828FBD1012196
:101DC00044F20D00FFF7C0FF01210220FFF7ACFF36
:101DD00010BD00000F48006840F001000D49086088
:101DE000084640680C4908400A49486008460068AF
:101DF0000A490840074908600846006820F4802026
:101E000008600846406820F4FE0048604FF41F0058
:101E100088607047001002400000FFF8FFFFF6FEE8
:101E200030B500210022002400232D4D6D6805F0FF
:101E30000C0121B1042905D0082923D105E0294D41
:101E4000056022E0274D05601FE0254D6D6805F413
:101E50007012234D6D6805F48034022505EB924223
:101E60001CB9214D554305600BE01D4D6D6805F40F
:101E700000351DB11C4D5543056002E0194D554319
:101E8000056002E0174D056000BF00BF144D6D688E
:101E900005F0F0010909154D6B5C0568DD404560F2
:101EA0000F4D6D6805F4E061090A104D6B5C4568E3
:101EB000DD4085600A4D6D6805F46051C90A0B4D1F
:101EC0006B5C4568DD40C560054D6D6805F44041BB
:101ED000890B074D6B5CC568B5FBF3F5056130BD3B
:101EE0000010024000127A0000093D00940000201A
:101EF000A400002010B501460022002300204A1152
:101F0000012A02D1094C236806E0022A02D1074CBB
:101F1000236A01E0054C636A01F01F02012494402A
:101F20001C400CB1012000E0002010BD0010024058
:101F30000248406800F00C007047000000100240AA
:101F400001460020034A506820F0F000084350602A
:101F500070470000001002401149096821F48031E7
:101F60000F4A11601146096821F480211160B0F513
:101F7000803F03D0B0F5802F0ED106E008490968F4
:101F800041F48031064A116007E00549096841F4CF
:101F9000A021034A116000E000BF00BF70470000AD
:101FA0000010024001460020034A506820F4E0601F
:101FB00008435060704700000010024001460020B6
:101FC000034A506820F4605040EAC10050607047F6
:101FD00000100240014908667047000000004242BC
:101FE00002460020044B586820F47C1042EA0103AA
:101FF0001843014B58607047001002400146002012
:10200000034A506820F00300084350607047000006
:102010000010024038B5002000900024002500BFC9
:102020003120FFF767FF05460098401C009000989C
:10203000B0F5A06F01D0002DF2D03120FFF75AFF8C
:1020400008B1012400E00024204638BD10B586B058
:102050000024142101A8FEF78EF80A2201A90848DD
:1020600000F012F800BF07E001A810F81400054ABC
:1020700002F81400601CC4B20A2CF5DB06B010BDD7
:10208000000003084C05002070B504460D461646B6
:10209000002300BF07E02046FEF7BEFF25F813002F
:1020A000A41C581CC3B2B342F5DB70BD00B587B0A9
:1020B000012141F20500FFF747FEE020ADF81800CE
:1020C00018208DF81B0003208DF81A0006A9164869
:1020D000FEF713FFE0211448FEF79CFF0020ADF847
:1020E00004004FF48270ADF806000020ADF808003F
:1020F000ADF80A00ADF80C004FF40070ADF80E001A
:102100001820ADF810000020ADF812000720ADF83F
:10211000140001A9054800F06BF80121034800F004
:102120004DF807B000BD000000080140003001403C
:1021300000B587B001218803FFF7F6FD01210920D2
:10214000FFF702FE4FF46040ADF8180018208DF83C
:102150001B0003208DF81A0006A91648FEF7CDFED5
:102160004FF460411348FEF755FF0020ADF804001E
:102170004FF48270ADF806000020ADF80800ADF80D
:102180000A00ADF80C004FF40070ADF80E001820F6
:10219000ADF810000020ADF812000720ADF81400D3
:1021A00001A9054800F024F80121034800F006F8D1
:1021B00007B000BD000C01400038004021B102888A
:1021C00042F04002028004E002884FF6BF731A40DA
:1021D000028070470246002013890B400BB101209A
:1021E00000E0002070470146888970478181704770
:1021F00010B50022028802F441520B884C88234318
:102200008C882343CC8823430C8923434C89234364
:102210008C892343CC8923431A430280838B4FF25A
:10222000FF74234083830B8A038210BD2DE9F041A4
:1022300006460F4626BB06E0601CC4B2C82C02DB73
:102240000020BDE8F08102212048FFF7C3FF0028ED
:10225000F2D039461D48FFF7C9FF002405E0601C95
:10226000C4B2C82C01DB0020EBE701211748FFF7BF
:10227000B1FF0028F3D01548FFF7B5FFC5B222E043
:1022800005E0601CC4B2C82C01DB0020D9E70221A4
:102290000F48FFF79FFF0028F3D039460C48FFF79F
:1022A000A5FF002405E0601CC4B2C82C01DB00209F
:1022B000C7E701210648FFF78DFF0028F3D0044847
:1022C000FFF791FFC5B22846BBE700000030014090
:1022D0000038004070B505460C467DB90F480088AF
:1022E0004FF6C77108400D49088008460088204312
:1022F000088001210A48FFF761FF0EE008480088C6
:102300004FF6C771084006490880084600882043F8
:10231000088001210248FFF751FF70BD00300140E5
:1023200000380040704770B504460D4629462046E7
:10233000FEF7A4FD70BD000010B586B00024142186
:1023400001A8FDF718FF00BF07E00B4830F81400A4
:1023500001A921F81400601CC4B20A2CF5DB07485F
:1023600000F0FEF80A2201A9044800F009F800F084
:1023700078FC06B010BD00003805002000000308FE
:102380002DE9F04105460F461646002400BF07E040
:1023900037F814102846FFF7C6FFAD1C601CC4B206
:1023A000B442F5DBBDE8F08170B504460D46034A42
:1023B0002946204600F028F870BD00000038014092
:1023C00010B504460249204600F00EF810BD00008A
:1023D0000044004010B504460249204600F02DF8A4
:1023E00010BD00000044004070B504460D4600BF1B
:1023F0008021284600F062FB0028F9D021462846BB
:1024000000F029FC012070BD2DE9F04104460D4685
:10241000164614B90120BDE8F0810AE014F8017BEA
:1024200031463846FFF7E0FF08B90020F3E7681EA1
:1024300085B2002DF2D10120EDE770B504460E46BD
:102440000CB9012070BD11E014F8015B0A2D06D112
:1024500031460D20FFF7C8FF08B90020F2E73146EA
:102460002846FFF7C1FF08B90020EBE720780028D5
:10247000EAD10120E6E710B500F002F810BD000037
:102480000CB50020019000903348006840F4803083
:102490003149086000BF3048006800F40030009007
:1024A0000198401C0190009818B90198B0F5A06FF0
:1024B000F1D12948006800F4003010B101200090EB
:1024C00001E0002000900098012843D123480068D3
:1024D00040F01000214908600846006820F0030021
:1024E00008600846006840F0020008601A4840682A
:1024F000194948600846406848600846406840F40A
:10250000806048600846406820F47C1048600846B7
:10251000406840F4E81048600846006840F0807069
:10252000086000BF0C48006800F000700028F9D077
:102530000948406820F003000749486008464068A1
:1025400040F00200486000BF0348406800F00C0003
:102550000828F9D10CBD0000001002400020024004
:1025600010B50446FEF7AAFC2046FEF73DFC10BD60
:102570007047000010B51348006840F00100114991
:10258000086008464068104908400E4948600846FF
:1025900000680E4908400B4908600846006820F4AE
:1025A000802008600846406820F4FE0048604FF430
:1025B0001F008860FFF75FFF4FF00060044908606C
:1025C00010BD0000001002400000FFF8FFFFF6FE03
:1025D00008ED00E010B50121204800F07EF8002849
:1025E0003AD001211D4800F069F81D480088401CC0
:1025F0001B4908801B480088401C1A4908801A485B
:102600000088401C1849088018480078C0B14FF471
:1026100000711748FEF7FEFC16480088401C15495B
:10262000088008460088B0F5C87F09DB4FF40071C8
:102630000F48FEF7EDFC00200E4908800B4908709A
:102640000948008841F28831884202D100200649B9
:10265000088001200849087010BD000000040040F7
:102660002000002032000020220000202500002051
:102670000010014026000020240000203EB5054641
:102680000C4601210220FFF74FFBADF80450ADF8D6
:1026900000400020ADF80600ADF80200694606488B
:1026A00000F036F801221146034800F027F8012116
:1026B000014800F006F83EBD00040040CA43028213
:1026C000704721B1028842F00102028004E00288D2
:1026D0004FF6FE731A400280704730B50246002064
:1026E00000230024158A05EA0103958905EA0104FF
:1026F00013B10CB1012000E0002030BD1AB1838974
:102700000B43838102E083898B4383817047000000
:10271000002202881D4B98420ED01D4B98420BD0D0
:10272000B0F1804F08D01B4B984205D01A4B98420D
:1027300002D01A4B984204D14FF68F731A404B883F
:102740001A43174B984207D0164B984204D04FF6C5
:10275000FF431A40CB881A4302808B8883850B88FD
:1027600003850A4B98420BD0094B984208D00E4B78
:10277000984205D00D4B984202D00D4B984201D1A2
:102780000B7A03860123838270470000002C0140EE
:10279000003401400004004000080040000C0040EC
:1027A000001000400014004000400140004401407F
:1027B0000048014010B540F22551124800F08BF955
:1027C00088B140F225510F4800F0CFF80D4800F0D5
:1027D0003DFAC4B20C480D49097844540B480078BE
:1027E000401C0A4908700821064800F067F90128D2
:1027F00006D10821034800F0AFF8024800F026FA9D
:1028000010BD00000038014010010020030000202E
:1028100010B540F22551124800F05DF988B140F240
:1028200025510F4800F0A1F80D4800F00FFAC4B28E
:102830000C480D49097844540B480078401C0A495B
:1028400008700821064800F039F9012806D108214E
:10285000034800F081F8024800F0F8F910BD0000CC
:1028600000440040F80400208500002010B586B028
:10287000044601210520FFF767FA01214804FFF70C
:1028800053FA0420ADF8140003208DF81600182028
:102890008DF8170005A91548FEF72FFB0820ADF8A5
:1028A000140004208DF8170005A91048FEF725FB39
:1028B00001940020ADF80800ADF80A00ADF80C0056
:1028C000ADF810000C20ADF80E0001A9084800F08A
:1028D00051F9012240F22551054800F026F9012165
:1028E000034800F051F806B010BD00000008014098
:1028F0000044004010B540F22551144800F0EBF8B8
:10290000B0B140F22551114800F02FF80F4800F007
:102910009DF9C4B20E480F49097844540D48007817
:10292000401C0C4908700846007800F00F00087041
:102930000821064800F0C2F8012806D10821034802
:1029400000F00AF8014800F081F910BD004800408D
:10295000D80100200900002001F40072B2F5007FC8
:1029600000D100BFCA430280704710B50022002387
:1029700040F66A14A14200D100BF0A12012494401B
:10298000A3B2DC43048010BD21B1828942F400521D
:10299000828104E082894DF6FF731A40828170477C
:1029A00000B585B0012144F20400FFF7CDF94FF4E2
:1029B0000070ADF8000003208DF8020018208DF89B
:1029C000030069463948FEF798FA4FF48060ADF885
:1029D000000004208DF8030069463448FEF78DFAA4
:1029E0004FF4164001900020ADF80800ADF80A0041
:1029F000ADF80C00ADF810000C20ADF80E0001A9E8
:102A00002B4800F0B7F8012240F22551284800F089
:102A10008CF801212648FFF7B7FF01218804FFF752
:102A200083F901210820FFF78FF94FF48060ADF89A
:102A3000000003208DF8020018208DF8030069467D
:102A40001C48FEF75AFA4FF40060ADF8000004206D
:102A50008DF8030069461748FEF74FFA4FF4965079
:102A600001900020ADF80800ADF80A00ADF80C00A8
:102A7000ADF810000C20ADF80E0001A90E4800F0D2
:102A800079F801A90C4800F075F8012240F22551AF
:102A9000094800F04AF801210748FFF775FF402177
:102AA0000348FFF759FF05B000BD000000080140D2
:102AB00000380140000C0140004800400246002060
:102AC000B1F5007F00D100BF13880B400BB101208E
:102AD00000E00020704770B5024600240023002566
:102AE000002040F66A16B14200D100BFC1F3421582
:102AF00001F01F03012606FA03F3012D02D1968986
:102B0000334006E0022D02D1168A334001E0968A56
:102B100033400C12012606FA04F41688344013B12F
:102B20000CB1012000E0002070BDF0B50346002488
:102B300000260025002040F66A17B94200D100BFE8
:102B40001846C1F3421401F01F06012707FA06F5E3
:102B5000012C01D10C3004E0022C01D1103000E036
:102B600014301AB107682F43076002E00768AF43CB
:102B70000760F0BD2DE9F04786B005460E460024FB
:102B8000A24600BFA1460027B08900B100BF2F4672
:102B90002C8A4CF6FF700440F08804432C82AC89E8
:102BA0004EF6F3100440B088318908437189084318
:102BB0000443AC81AC8A4FF6FF400440B089044323
:102BC000AC8201A8FFF72CF91F48874202D1DDF83B
:102BD00010A001E0DDF80CA0A88900F4004040B18D
:102BE0000AEBCA0000EB0A1031684900B0FBF1F8AB
:102BF00007E00AEBCA0000EB0A1031688900B0FB5D
:102C0000F1F86420B8FBF0F004012009642101FB15
:102C10001089A88900F4004040B1322000EBC900BF
:102C2000B0FBF1F000F00700044308E0322000EBB5
:102C300009106421B0FBF1F000F00F0004432C8177
:102C400006B0BDE8F08700000038014001468888E2
:102C5000C0F308007047C1F308028280704700BFCC
:102C6000FEE710B5FEF700F910BD0000014A024969
:102C700000F013B8392E0008A800002002E008C8B0
:102C8000121F08C1002AFAD170477047002001E0E6
:102C900001C1121F002AFBD170472DE9F0411646F1
:102CA0000F460446002503E03946B047641C6D1CFE
:102CB00020780028F8D12846BDE8F08170B5054697
:102CC0000C4605F1B001C8B20749096888471021D0
:102CD00001EB241004490968884704F00F000249F9
:102CE0000968884770BD00008C00002010B54FF4C3
:102CF00080511E48FEF78EF904211C48FEF788F922
:102D00004FF480611948FEF785F9002421E04FF463
:102D100000611648FEF77CF91548007800F0800045
:102D200028B94FF480511148FEF772F904E04FF4CE
:102D300080510E48FEF76EF90D4800784006000EEF
:102D40000B4908704FF400610848FEF763F9601CF6
:102D5000C4B2082CDBDB04210448FEF75BF94FF416
:102D600080510248FEF756F910BD000000100140E6
:102D70008800002070B5044600BF4FF480511B4806
:102D8000FEF748F904211948FEF742F94FF4806133
:102D90001648FEF73DF900251BE04FF4006113488B
:102DA000FEF736F904F0800028B94FF480510F483F
:102DB000FEF72EF904E04FF480510C48FEF72AF993
:102DC0006006040E4FF400610848FEF723F9681C02
:102DD000C5B2082DE1DB04210448FEF71BF94FF4CE
:102DE00080510248FEF716F970BD00000010014046
:102DF000014605E0122001E0421E90B20028FBDCF3
:102E00000A00A1F1010399B2F4D1704710B502464E
:102E10000BE0C82007E0122101E04B1E99B2002907
:102E2000FBDC431E98B20028F5DC1300A2F101047C
:102E3000A2B2EED110BD000070B504460D46E0B25E
:102E40000549088000BF40210348001FFFF736FEF8
:102E50000028F8D0204670BD0438014008B5012094
:102E6000ADF8000010208DF8030003208DF802005B
:102E700069461A48FEF741F80420ADF8000069469B
:102E80001648FEF73AF80820ADF8000069461348E6
:102E9000FEF733F84FF48060ADF8000069460F4844
:102EA000FEF72BF84FF40060ADF8000069460B48C0
:102EB000FEF723F84FF48050ADF80000694607484C
:102EC000FEF71BF801210548FEF7A4F818210020A1
:102ED00000F05EF900F036F908BD00000010014076
:102EE00008B501211020FEF72FFF0120ADF80000EA
:102EF00010208DF8030003208DF8020069460D486C
:102F0000FDF7FBFF01210B48FEF784F84FF400703A
:102F1000ADF8000010208DF8030003208DF80200AA
:102F200069460448FDF7E9FF4FF400710148FEF7D8
:102F30006FF808BD00100140FEF716FFFEF772FEA5
:102F400040F271210420FEF789F8FEF783F841F67C
:102F50001F410920FFF792FBFFF7C2FFFFF77EFF3B
:102F6000FFF71EFD4FF4E130FFF780FCFEF7D2F8CB
:102F7000FEF770F802E03BA0FFF778FE0120FEF7B5
:102F80009DF80028F7D1FDF773FEFEF763F8394886
:102F90000068C0433849C1F88001C820FFF736FFF8
:102FA0003548D0F88001C0433349C1F8800106217B
:102FB00032A0FDF7FEFE33A0FFF70CFAFEF74AF849
:102FC00031A0FFF753FE0120FEF73EFAFFF73EF86F
:102FD0003448007834490870084600780C2837D205
:102FE000DFE800F0060A0E12161A1E22262A2E32DA
:102FF0002EA0FFF73BFE2BE02FA0FFF737FE27E0C8
:1030000030A0FFF733FE23E031A0FFF72FFE1FE0D3
:1030100032A0FFF72BFE1BE033A0FFF727FE17E0DF
:1030200035A0FFF723FE13E036A0FFF71FFE0FE0E9
:1030300037A0FFF71BFE0BE038A0FFF717FE07E0F5
:1030400039A0FFF713FE03E03AA0FFF70FFE00BF21
:1030500000BF3220FFF7DAFE03E0FDF7BDF8FDF711
:1030600001FBFAE754686520322E3447204572721E
:103070006F7221008001224200002242313233343B
:10308000353600000A0000000A5043B6D4C2EBC82F
:10309000EDBCFECDA8D3C3B0E6B1BE56312E370A83
:1030A000000000004C0500202A000020BDADCEF736
:1030B000D0ADD2E90D0A0000CCECB2A8D0ADD2E977
:1030C0000D0A0000D4C6C4CFD0ADD2E90D0A00006D
:1030D000B9F3D6DDD0ADD2E90D0A0000CBC4B4A857
:1030E000D0ADD2E90D0A0000C4DAC3C9B9C5D0AD6C
:1030F000D2E90D0A00000000B0B2BBD5D0ADD2E9D4
:103100000D0A0000C9BDCEF7D0ADD2E90D0A00000E
:1031100056434F4DB2E2CAD40D0A0000C1C9C4FEE5
:10312000B5E7D0C50D0A0000C1C9C4FED2C6B6AF0E
:103130000D0A00005470D7A8D3C3D0ADD2E90D0A50
:103140000000000070B5002411E000200D49087057
:1031500000212046FFF7B2FD002504E00A48006880
:103160008047681CC5B2852DF8DB601CC4B2082CF2
:10317000EBDBAF200549096888472F200349096820
:10318000884770BD88000020900000208C0000203F
:1031900070B504460D4605480549086005480649CE
:1031A00008602946204600F009F870BD752D00081A
:1031B0008C000020ED2C00089000002070B5054622
:1031C0000C4605B34FF480513048FDF723FF012032
:1031D000FFF70EFE08212D48FDF71CFF04212B48A8
:1031E000FDF716FF0520FFF711FE08212748FDF720
:1031F0000FFF1E20FFF70AFE08212448FDF70AFFF3
:103200001320FFF703FE04212048FDF701FF4FF4D0
:1032100080511E48FDF7FEFE08211C48FDF7FAFE0E
:10322000A2201B4909688847A020194909688847D6
:10323000C820174909688847A620154909688847A2
:103240002F201349096888470220FFF7D1FDF82095
:103250000F490968884701200D49096888472420DB
:103260000B4909688847242481200949096888474F
:103270002046074909688847AF20054909688847FB
:10328000602003490968884770BD000000100140B4
:103290008C000020344310100134431010013320FF
:1032A0000D547933200D547934431010010110105E
:1032B00043343223ABBA013412BBAA0134128675EF
:1032C000014656431000346E46100134431010017D
:1032D000862C95010136E4A7BC014218BAE801002A
:1032E0000033000800000020AC0000007C2C000827
:1032F000AC330008AC000020545F00008C2C0008A8
:10330000000000000000000000000000D1D1E0D06B
:1033100000000000D2D20000000000000000000009
:10332000000000000000000000000000000000009D
:10333000000000000000000000000000000000008D
:1033400000003132333435363738393132333435A1
:10335000363738390000000000000000000000008F
:103360000000313233343536373839313233343581
:10337000363738390000000000000000000000006F
:10338000000000000000000000000000000000003D
:103390000000000000000000010203040102030419
:0C33A000060708090204060800000000EF
:0400000508000131BD
:00000001FF
